:10000000DAC00000F5C00000F3C000000C94FA0D47
:10001000EFC00000EDC00000EBC000000C94E90D43
:10002000E7C00000E5C00000E3C00000E1C0000040
:10003000DFC00000DDC00000DBC00000D9C0000050
:10004000D7C00000D5C00000D3C00000D1C0000060
:100050000C947C0DCDC00000CBC00000C9C00000D6
:10006000C7C00000C5C00000C3C00000C1C0000080
:10007000BFC00000BDC00000BBC000003230323243
:1000800030373032303731340000000000000000DB
:100090000000000000000000000000000000000060
:1000A0000000000000000000000000000000000050
:1000B0000000000000000000000000000000000040
:1000C0000000000000000000000000010203040521
:1000D000060708090A0B0C0D0D0F10111213151647
:1000E00017191A1B1C1E202122242627292A2C2EF0
:1000F0002F31333537393B3D3F41434547494B4E1F
:10010000505254575A5C5E616366686C6E717477C6
:10011000797D7F8286888C8F9295999C9FA3A6017A
:100120000102020303040405060708090A0C0D0E68
:100130000F11131416181A1D1F2224272A2D3033CD
:10014000373B3E42464B4F54595D63686E73797F2F
:10015000868C939AA1A8B0B8C0C8D1D9E2ECF5FFBB
:10016000FFFFFFFFFFFFFFFFFFFFFFFFFFFFFFFF9F
:10017000FFFFFFFFFFFFFFFFFFFFFFFFFFFFFFFF8F
:10018000FFFFFFFFFFFFFFFFFFFFFFFFFFFFFFFF7F
:10019000FFFFFFFFFFFFFFFFFFFFFFFFFFFFFFFF6F
:1001A000FFFFFFFFFFFFFFFFFFFFFFFFFFFFFFFF5F
:1001B000FFFFFFFFFF0011241FBECFEFCDBFDFE326
:1001C000DEBF18E3A0E0B8E3EAEAF2E202C005907D
:1001D0000D92A032B107D9F728E3A0E2B8E301C03D
:1001E0001D92A83CB207E1F70E940A0E0C94481138
:1001F00007CFF89498ED94BF8093610080916300DD
:1002000080FDFCCF78940895E5E9F8E320E030E044
:100210009081992339F02F5F3F4F3396203131057C
:10022000B9F70BC0F901EE0FFF1F2E0F3F1FF901A9
:10023000EB56F74C80836183728308950F931F936D
:10024000CF93DF93D0919538DD2351F1009196380B
:1002500010919738C0917238C150C7FD0DC0EC2F76
:10026000EE0FFF0BED58F74C0190F081E02DB80137
:100270008D2F09958111F0CFE5E9F8E38381808323
:100280008481958181839283339688E3E23CF807E9
:10029000A9F71092C2381092C3381092C438D2CF46
:1002A000DF91CF911F910F910895BC018091C738C4
:1002B000ABCF1092C7381092C5381092C63881E083
:1002C00080934C3808950F931F93CF93C82F02E962
:1002D00019E0CC2349F085E08CDFC8010197F1F7E4
:1002E00081E087DFC150F5CFCF911F910F91089525
:1002F000E0E0F6E08285816082878085816080878A
:10030000089582B185FB882780F991E08927809341
:100310006B380895E0910638F09107383196FB70FC
:10032000F460E0930638F0930738809167388B5A71
:1003300080936738E491809167388E0F0895882301
:1003400049F0813069F480E28093220488E0809350
:100350003504089580E28093210480932604089553
:1003600080E280932104809325040895CF93C82FC1
:10037000809369388093683880916A38811101C010
:10038000DEDFC11109C010922A0A10922B0A1092C6
:10039000280A1092290A17C08FEF8C0F90E0FC01F9
:1003A000E15EFE4FE491F0E0E0932A0AF0932B0A1D
:1003B000FC01E757FF4FE491F0E0E093280AF09347
:1003C000290AC53010F485E005C0CE3010F483E072
:1003D00001C081E0CF910DCFCF93DF93CDB7DEB7D2
:1003E0002697CDBFDEBF909147382091833830915A
:1003F0008438295B394009F492E0843019F4609321
:1004000048381FC06623E9F0823019F427E9261B1B
:10041000622F26E0E4E9F2EADE01119601900D92E6
:100420002A95E1F79E012F5F3F4F280F311D280FBE
:10043000311DF90132970190F081E02DE90FF11D96
:1004400060832696CDBFDEBFDF91CF910895BF9226
:10045000CF92DF92EF92FF920F931F93CF93DF9390
:10046000EC0140914738E0911A38EE2311F082E018
:1004700001C0842F90E0DC01AC5EB74C2C9120933E
:100480001838DC01AF5EB74C8C9180931738F0E0E0
:10049000E25FF74C3181622F70E0442349F0313044
:1004A00039F49B01280F311DC9019595879538C0F6
:1004B000C617D707A4F1682F70E06C177D0784F189
:1004C000411102C08C2F2CC0821B032F10E0015061
:1004D0001109E82EF12CC701B8010E9401116093A7
:1004E00045386695E62FF0E0822FC12CD12CB12C37
:1004F000B316B1F0C601B8010E94ED10822F860F2D
:10050000CE0CDF1CAE01481B510957FF03C05195AB
:1005100041955109E417F5071CF4B394E9CF822FF4
:10052000DF91CF911F910F91FF90EF90DF90CF90CF
:10053000BF90089580934B3819CFCF93C0916938FD
:1005400089E18C0F873908F080E010DF82E0BBDEA4
:100550008C2FCF910BCFCF93C091693880E006DF0D
:1005600083E0B1DE8C2FCF9101CF81E0089561113E
:1005700060931D380895662389F0813061F480917D
:10058000863890918538891B681B6093853882E096
:1005900080931E3803C0635E60931C3880911C38C2
:1005A000873418F086E480931C38089560934038AF
:1005B00008950F931F93CF93DF93809147388093D3
:1005C0004D388091143880934E3880911138809343
:1005D0004F3880910E388093503880911538809331
:1005E0005138809112388093523880910F3880931F
:1005F0005338809116388093543880911338809303
:100600005538809110388093563880911A388093ED
:100610005738809148388093583880914638809375
:1006200059388091193880935A3880914A3880938C
:100630005B388091493880935C3880910B38809387
:100640005D388091093880935E3880910A388093B4
:100650005F38809108388093603880910C3880939F
:10066000613880911C3880936238809185388093FE
:10067000633880911D388093643880910D38809361
:1006800065388091403880936638F8940DE418E31B
:10069000C1E4D0E0F80161918F01CE010E942B11DD
:1006A0002196CB35D105B1F765EA80E490E00E9450
:1006B0002B117894DF91CF911F910F910895109293
:1006C00094389091100680916738890F809367382D
:1006D00080918938882309F419C110928938909142
:1006E000923880916A38882339F0809100068E7F95
:1006F0008093000610929238911143C080911E3869
:10070000882349F060918E3870918F3860938A38D1
:1007100070938B3804C060918A3870918B38605F19
:100720007F4FA6E076956795AA95E1F780E098E57A
:100730000E94ED1080911D3890E00297680F791F9C
:10074000769567956093883880913C38882311F0BE
:10075000815007C06D3138F460E070E084E054DD12
:1007600085E080933C3880916A388111C6C08EE163
:100770008093060685E48093020681E08093923898
:10078000B9C0913009F0B9C080911E38811143C0C1
:1007900080918C3890918D3840969C0145E036953B
:1007A00027954A95E1F7A0918538A9015695479577
:1007B0000A2E000CBB0BCD0183519140840F951F75
:1007C000809386389093873880912B38E82FF0E01B
:1007D000EE0FFF1FE45DF74C40815181B901641BAE
:1007E000750B208331838F5F877080932B38CB010B
:1007F000880F991F880F991F40911C3850E04D5E5B
:100800005E4F4A1B5B0B440F551F841B950B820FD9
:10081000931F23E01CC08091903890919138809371
:100820008C3890938D38409635E0969587953A951B
:10083000E1F7ECE2F8E38193919328E3EC33F207DC
:10084000D1F7A6CF009709F00196215029F018168C
:100850001906C4F70197F9CF18161906E4F477FDC5
:1008600039C020912A3812160CF1880F991FBC014B
:100870006350710977FF02C06F5F7F4F7595679571
:100880001616170614F061E070E088E1861B80936D
:100890002A3885E026C08C3F2FEF9207DCF477FFE3
:1008A00019C020912A3827FF05C02450281B209307
:1008B0002A3818C024EE281B20932A382091883823
:1008C0002F3180F06CEF7FEF681B790B7595679582
:1008D00086E007C0809188388E3120F060E070E0BB
:1008E00087E092DC8DE18093060685E58093020621
:1008F0001092923810929338FBDC80911E38882336
:1009000029F080911E38815080931E3808958130DF
:1009100019F410924A380895823019F460934938D6
:100920000895833019F4609346380895843011F4A3
:10093000609319380895909188389D3110F480E0C3
:1009400006C08F70E82FF0E0E656FD458081F7CCB9
:10095000CF93C0911A38C1114AC0883039F410922F
:100960004438109241381092423842C0813B59F4C9
:100970008091443881508330D0F583E080934438AF
:100980008093433834C0853BB1F4CB016EE370E013
:100990000E94ED10892B61F5809144388A3F40F523
:1009A0008B5F809344388093433810924138109283
:1009B0004238C3DD1DC08130D1F48091413890911F
:1009C0004238019688382EE0920728F48093413807
:1009D000909342380DC01092413810924238809165
:1009E0004438882329F081508093443801C0C1E005
:1009F0008C2FCF910895FF920F931F93CF93DF9386
:100A00008C01EB01F42E8091833890918438892BEE
:100A100031F0E0918338F091843889E009950093B2
:100A2000833810938438012B39F0E0918338F091AA
:100A30008438BE018F2D099581E080934C38DF9179
:100A4000CF911F910F91FF900895CF93DF93E09185
:100A50007238EE2359F0E150E0937238F0E0EE0F77
:100A6000FF1FED58F74CC081D18102C0C0E0D0E03B
:100A7000E0917238EE2341F0F0E0EE0FFF1FEF58E7
:100A8000F74C8081918102C080E090E04AE060E014
:100A900070E0B1DFCE01DF91CF910895883029F465
:100AA00010923D381092243815C08130F9F490919D
:100AB0002438911107C06032710568F180932438A1
:100AC000F8DB29C0913081F46B3B710528F082E09E
:100AD0008093243880E01EC061157105E1F06270DA
:100AE000862F880F8E5E16C0B0DF15C0813811F0DA
:100AF000813E89F491E090932438813E21F48091E5
:100B00003D38865F03C080913D388F5F80933D38CC
:100B1000D0DB8BE42BDC80E008959C01909172384F
:100B2000983088F4E92FF0E0EE0FFF1FED58F74CF6
:100B3000208331839F5F9093723848E0C9015BDF67
:100B40008091723808958FEF08950F931F93CF937C
:100B5000DF93EC018B0179DFB801CE01DF91CF91FA
:100B60001F910F91DACF813C29F460E070E08EE4B0
:100B700096E006C0823C39F460E070E084E196E0E3
:100B8000E4DF80E0089581E00895843011F58091DC
:100B90008338909184382BE08D3A920729F469E1EB
:100BA00070E082E397E013C08253974061F4909124
:100BB0006938923040F0892F869596959695890FE1
:100BC000B9DC80E0089560E070E08EE496E0BDDF7F
:100BD000F8CF81E00895813C29F460E070E08EE474
:100BE00096E006C0823C31F460E070E083EB95E073
:100BF000ACDF16C0813B49F4CB016EE370E00E948C
:100C0000ED10892B69F499DC0BC0813E59F4CB01BE
:100C10006EE370E00E94ED106F5F60930C38C9DCEA
:100C200080E0089581E00895CF93C0911A38C111F2
:100C300017C0813C29F460E070E08EE496E006C0C5
:100C4000823C31F460E070E084E396E07EDF09C02E
:100C5000873B31F460E070E081EC99E05EDF01C039
:100C6000C1E08C2FCF910895813C29F460E070E0C1
:100C70008EE496E006C0823C31F460E070E08BEEDA
:100C800095E063DF07C0873B39F460E070E085ECF6
:100C900099E043DF80E0089581E008950F931F936A
:100CA000CF938B01883079F480E060DB80910D3840
:100CB000837045DB10924438012B19F481E0809356
:100CC0006A38C0E0CAC0813051F469317105C8F397
:100CD00080936A3880910D38837031DBF2CF833096
:100CE00041F580914A38882371F09091493842EC5F
:100CF00051E0949F9001959F300D11246217730766
:100D000010F080931B3880910D388370833011F47C
:100D1000802F11DE80914038882399F242EC51E017
:100D2000849F9001859F300D11242017310748F6CC
:100D30004DC0813B99F481E090E089DB17DB809125
:100D400046388111BECF80914738811104C00831E7
:100D5000110508F4B6CF61E070E028C0813ED9F3F8
:100D6000813821F480911B3890E013C0813C21F43C
:100D70006091693870E01AC0823B79F4809119382B
:100D800090911A38911180914838811104C086E9F8
:100D900090E05DDB05C086E903C0823E19F480E087
:100DA000E5DA8FCF823C31F466E970E082E397E0C8
:100DB000CCDE87CF833999F3833C29F460E070E07F
:100DC00084E196E0F5CF843C31F4B7DB60E070E07D
:100DD0008DEC99E0EDCF8F3C29F460E070E085EB7D
:100DE00092E0E6CFC0911A388A3B79F4672B69F418
:100DF000CC2329F0A2DB10921A38DBDB62CF60E053
:100E000070E089EB99E089DE28C0C11125C08A3CD9
:100E100029F493DB81E080931A381CC0833B29F4CA
:100E200060E070E08DEA9BE007C0853C39F485DB2B
:100E300060E070E085E39DE088DE0FC0873C61F4F0
:100E400090910D3881E0890F83709C7F982B90934F
:100E50000D3875DAAEDB01C0C1E08C2FCF911F9148
:100E60000F9108959F92AF92BF92CF92DF92EF922F
:100E7000FF920F931F93CF93DF93182FEB01D09026
:100E80001838F0901738A0904738AA2019F0B09081
:100E9000453802C0BB24B394C090193800911A3869
:100EA0000111C0904838CC2051F041E0C41621F027
:100EB00080911B388F1518F0F6E9EF2E01C0EF2C4A
:100EC00090904438BE01812F43DD20914438222385
:100ED00039F091100CC0809169388093283807C090
:100EE000992029F060E070E08EE496E039C0812F0F
:100EF0008D7F8830D9F410923F381A3019F4C091A0
:100F00001B38D0E08D2D90E08C179D0738F48F2D85
:100F100090E0C817D90710F4C0931B38CE0197DAB8
:100F200009DB81E08093053800E0D0C1113CD1F2AB
:100F3000123C71F4809169388E1510F48E2D02C028
:100F400080911B38F7DA8091693880932838ECCF8C
:100F5000143C41F480E00ADA60E070E08DEC99E046
:100F6000F4DDE2CF8FE4810F823008F04FC0AA2079
:100F700041F0CE0168E170E00E94ED10892B31F064
:100F8000D3CF60910E3870E0CE01F6CF80916938F2
:100F9000209761F4123B11F48FEF05C08F15E0F735
:100FA000D81648F181E08093053825C020910E388D
:100FB00030E066E371E0269FA001279F500D369F29
:100FC000500D11244C175D0710F48F1528F76CE6AF
:100FD00072E0269FA001279F500D369F500D1124CF
:100FE0004C175D0740F4D81630F0A7DA60E070E0E7
:100FF0008DEC99E0AADD30910538209169384B2DB0
:101000003403C0011124820F911D26C18FE1810F8D
:10101000823020F480910538819584CF113009F019
:10102000CEC0A99711F4109305382223B1F0409156
:10103000283830E021503109429FC001439F900D74
:1010400011246091433870E00E940111611101C0C8
:1010500061E06093683860934B38C0916838309194
:1010600069388C2F90E0831B91096091263870912C
:1010700027386F5F7F4F609326387093273800972B
:1010800009F452CF97FF05C0333830F040E450E008
:1010900005C040E052E002C040E051E0569547955F
:1010A00097FD0196959587950097C1F746175707C5
:1010B00008F03ACFC31710F48FEF03C03C1718F4B1
:1010C00081E0830F01C08C2F9FEF980FA92FB0E014
:1010D000AD01415E5E4FFA016491931778F420915F
:1010E0002A0A30912B0A232B49F46F3F39F42FEF52
:1010F00030E020932A0A30932B0A20C020912A0A3C
:1011000030912B0A70E02617370738F460912A0ACD
:1011100070912B0A6F5F7F4F0DC020912A0A30918A
:101120002B0A6217730750F460912A0A70912B0AF8
:101130006150710960932A0A70932B0A9D01275709
:101140003F4FF9016491E091280AF091290A70E07B
:10115000E617F70738F46091280A7091290A6F5F43
:101160007F4F0DC0E091280AF091290A6E177F0782
:1011700050F46091280A7091290A615071096093B6
:10118000280A7093290A60912A0A70912B0AFA01A1
:10119000449150E06417750769F44091280A509112
:1011A000290AF901249130E04217530719F4DED8D7
:1011B000C09368381092263810922738B5CE153073
:1011C000A9F480916938823408F4AECE90E08C1B8B
:1011D0009D0B282F813491052CF08739910518F04B
:1011E00026E901C021E4209368389ECE1630B9F478
:1011F0009091693880914B38981708F095CEC90FB7
:10120000D11D90E08C179D0734F0C134D10524F432
:10121000C1E4D0E001C0EC01C093683885CE17303E
:1012200079F49091683880916938891710F48F5F4C
:1012300004C0981708F078CE81508093683874CE37
:10124000133C71F481E0A11080E080934738B1D95C
:1012500082D98091693890E0FAD880931B3872CE99
:10126000011133C0133B49F4CD2B09F05DCECC20E6
:1012700011F086E9E82E8E2D04C0133E21F48091F2
:101280001B3858D923C0153C41F480E06FD860E08A
:1012900070E085E39DE059DC19C0173B29F460E05C
:1012A00070E085EB99E00FC01A3C39F48091693801
:1012B00080934A387ED941D909C01A3B31F460E0A5
:1012C00070E08DEB99E029DC01C001E0802FDF9117
:1012D000CF911F910F91FF90EF90DF90CF90BF9033
:1012E000AF909F900895883061F41092253880E087
:1012F0003DD880916B38811136C081E080932538CC
:1013000022C0982F907F903BB1F42091253842174E
:1013100078F0CB016DE570E060D7029739F42F5F6C
:10132000209325384217F8F088E303C082E101C01A
:1013300080E01CD818C0903E61F480912538882345
:1013400089F0481778F060E070E08EE495E0E5DB26
:101350000AC08A3041F460913D3880912538F90106
:10136000099527D972DB80E008952CEE31E043E047
:10137000BACF2CEE31E044E0B6CF27E834E044E0C9
:10138000B2CF27EB32E041E0AECF2BEB32E042E0D0
:10139000AACF26ED32E041E0A6CF0F931F93CF9363
:1013A000DF93D82F8B0180798039B9F420911438DC
:1013B000909115388D2F8F70823041F480914A388A
:1013C000811108C0822F291728F403C0822F921799
:1013D00008F4892F0E94B6011EC0803821F480E0F5
:1013E0000E94B60109C0D83039F480910D38869535
:1013F00086950E949F0142C0D13069F409311105E0
:1014000008F45CC0D0936A3880910D388695869533
:101410000E949F0153C0D33049F480910D388C70E5
:101420008C3009F04BC0802F86DA48C0D33C31F4B1
:1014300084D860E070E08EE496E00AC0D43C89F481
:10144000C0914A38CC2331F06C2F70E082E397E0F2
:101450007CDB34C060911B3870E082E397E075DB81
:1014600030C0D43B31F477D81092C73861E070E0D7
:10147000EDCFD53C19F466E970E0E8CFC0911A3899
:10148000C1111EC0DA3B31F460E070E089EC99E0F4
:1014900044DB17C0D73CA1F490910D38892F869575
:1014A00086958F5F8370282F220F220F9370920FE3
:1014B00090930D380E949F017CD803C0C0E001C00A
:1014C000C1E08C2FDF91CF911F910F910895CF93A1
:1014D000DF93C0E0D6E08DE18E8385E58A831092AC
:1014E0009238109293380E947801E0EAF0E080810F
:1014F0008061808383E08883888581608887DF912D
:10150000CF9108950F931F93CF9310926D388091D0
:10151000C5389091C6389C012F5F3F4F882790783F
:10152000822B932B8093C5389093C638C0916B382B
:101530000E948101C81731F110926A3880936B388C
:101540009091C738882359F0892F80699F709F3008
:1015500009F08F5F8093C73880E090E00DC0892F3D
:101560008F7E95FD02C0806801C0806C8093C73873
:101570008091C5389091C6380E9455011092C538A7
:101580001092C6380091C5381091C63880916A38DB
:10159000882379F0B80183E00E9404010E941E01B3
:1015A0000F731127012B09F043C0109229388FDFE8
:1015B00032C0C091C7388C2F807F803B19F460E027
:1015C00070E001C0B80181E00E940401C4FF13C0B3
:1015D000C5FF02C0C8010CC008311105E0F010922F
:1015E000C5381092C638C062C093C73880E090E01A
:1015F0000E94550110C0CC2371F0C5FD0AC0023114
:10160000110548F0C064C093C73880E090E00E94A4
:1016100055010E945901C0912938C11105C00E948D
:10162000780181E080938938CF5FCF71C0932938EA
:10163000CF911F910F9108958091943881113FD8D7
:1016400080916D3881115ECF0895EF92FF920F93D4
:101650001F93CF93DF93EC010AEC18E082E3E82EAE
:1016600082E0F82E2097D9F080914C38811119C072
:1016700080916938853028F485E00E94F900C7011F
:1016800004C081E00E94F900C8010197F1F781E0F0
:101690000E94F900D1DF0E941E012197E3CF81E073
:1016A00001C080E0DF91CF911F910F91FF90EF90EB
:1016B0000895CF93C82F882391F089E10E94B60145
:1016C00086EA90E0C2DF80E00E94B6018AEF90E0F7
:1016D000BCDFC15091F78AE992E0CF91B6CF89E1A2
:1016E0000E94B60188E090E0B0DF80E00E94B60181
:1016F0008AEF90E0AADFEFCFCF93DF9364E661D566
:10170000282F892F6AE05DD5EC01222341F0822F3A
:10171000D0DF8C2FCEDF8D2FDF91CF91CACFC111BB
:10172000F8CFF9CFCF93DF93D82FC3E080911B3848
:101730000E94B60188EC90E088DFDD2319F080E993
:1017400091E083DF80E00E94B60188EC90E07DDFCD
:10175000C15061F7DF91CF910895DF92EF92FF9230
:101760000F931F93CF93DF93D82F8B01C0910B382A
:1017700081E080933F38C33009F0E2C0F0904438F4
:101780008D2FE6D8FF2051F080914438811106C09A
:1017900060E070E08EE496E0D8D9D2C0D83021F471
:1017A00081E080930338CEC0D23C19F410924438C3
:1017B000D7C0D13BC1F490910238012B49F49E3639
:1017C00010F08FEF03C0923018F481E0809303385B
:1017D00080910338890F11F481E03CC18F3608F401
:1017E00039C18EE637C1D13E31F4809103388195FD
:1017F00080930338ECC0D23B61F481E080930338DE
:1018000080910238823008F4EAC081508093023817
:10181000E6C0D13009F0F4C00932110511F4D093BB
:101820000338D09023388D2D880FD7FC809527E082
:10183000829FC0011124E09022382E2D220FE7FC58
:101840002095D09101382D9F90011124232F290F2D
:10185000F09021388F2D880FF7FC8095C0910038CB
:101860008C9FC0011124822F890F6091023870E093
:10187000680F711D809144388130B9F480914138EE
:101880009091423825E0969587952A95E1F724E7CF
:1018900030E0A901481B590B469FC001479F900D9E
:1018A000569F900D1124B90198D4862F0E94B6013D
:1018B00000FD06C00E948A018170D80ED0922338A4
:1018C00080912038E80EE09222380E948A0165E279
:1018D00078D4F90EF09221380E948A018F7331F486
:1018E0000E948A016DE06DD490932038DD2339F099
:1018F0000E948A018F7319F4D150D09301380E944D
:101900008A01811108C00E948A016BE05AD4909329
:10191000013810922238C33038F00E948A018F714A
:1019200019F4C150C09300380E948A018F7709F0E2
:101930007CC00E948A0166E044D49093003875C050
:10194000D83021F481E08093043886C0D13C31F452
:1019500060E070E08EE496E0F8D87EC0D23C49F4B6
:101960008C2F90E0019665E070E04BD480930B38AB
:101970004CC0D13B51F5C23090F400FD6DC0EC2F4E
:10198000F0E0E75FF74C808190910438891B883044
:1019900020F08F3F99F58EEF31C088E02FC0C43022
:1019A00009F05AC09091083880910438890F82302C
:1019B00010F482E003C0893708F088E78093083884
:1019C000809108380E94B60147C0D13E31F4809121
:1019D000043881958093043818C0D23BA1F481E08B
:1019E00080930438C23068F500FD36C0EC2FF0E07B
:1019F000E75FF74C80818F3F79F18F5F80832CC048
:101A0000D13C09F4A5CFD23E19F40E94D90224C0DA
:101A1000D53C39F460E070E085E39DE096D880E045
:101A2000D1CFD13011F081E018C00932110519F47D
:101A300081E08093043880916738080F00936738FD
:101A40000BC0C43049F480910838833008F4B8CF13
:101A50008150B4CF8093023880E0DF91CF911F9105
:101A60000F91FF90EF90DF9008950F931F93CF9306
:101A7000DF93D82F8B01883031F480913F3881304B
:101A800011F488E06ADE8D2F8079803961F481E07D
:101A900080933E38C0913F38C1110CC080911B38F3
:101AA0000E94B60123C0803839F410923E3880E09D
:101AB0000E94B601C0E01AC0D130B9F4C0913E38DE
:101AC000CC2351F080913F388130A1F7B801DF91EC
:101AD000CF911F910F9141CE0733114058F3D0930E
:101AE0006A3880E00E949F0101C0C1E08C2FDF9125
:101AF000CF911F910F9108951F920F920FB60F92E1
:101B000011242F933F934F935F936F937F938F9302
:101B10009F93AF93BF93EF93FF9381E080930B0666
:101B200080919338882309F440C0E0919238E130E5
:101B3000D1F48091211120912011A0911006B09133
:101B40001106A81BB10987FDB39530E06DD3DC0108
:101B5000CB0180589F4FAF4FBF4F892F9A2FAB2F8C
:101B6000BB27BC0104C0609110067091110686E08D
:101B7000660F771F8A95E1F7F0E0EE0FFF1FDF0198
:101B8000A257B74C6D937C93E657F74C80819181B7
:101B90008617970708F401966817790708F40197E4
:101BA0008083918381E08093943881E0809393389F
:101BB000FF91EF91BF91AF919F918F917F916F9125
:101BC0005F914F913F912F910F900FBE0F901F90FB
:101BD00018951F920F920FB60F9211248F9381E0E8
:101BE0008093530180936D388F910F900FBE0F90AB
:101BF0001F9018951F920F920FB60F9211248F937A
:101C00001D9A81E080936C388F910F900FBE0F90DA
:101C10001F901895F89480914000877F8093400032
:101C200088EDA89584BF90910001907F909300016A
:101C300021E030E084BF2093610083E284B988E032
:101C400080931004809311048093120480931304F2
:101C50008093140499E09093150480931604809364
:101C60001704809332048093330480933404809368
:101C7000500480935104809352048093530487E36B
:101C80008093010A8FEF90E08093260A9093270AB1
:101C900091E09093000A8091120481608093120475
:101CA00090935201809151018111FCCF81E4809386
:101CB00050010DDC789481E00E94630160E070E0E7
:101CC00085EC95E00E948D0510924C380E949D0293
:101CD0000E948101811108C0F89480E490E0B3D2A1
:101CE000853AA9F17894A9C0C0E08C2F0E94B60172
:101CF00083E190E0AADC8C2F86950E94B60183E1F7
:101D000090E0A3DC0E9481018823B9F0CF5FC0344A
:101D100061F76091863880918538681B81E00E9468
:101D2000BB020E94D902C6E98C2F0E94B60184E052
:101D300090E08BDCC150C1F7CFCFCC2369F28C2F60
:101D40000E94B6018DE090E080DCC150F6CF0DE43A
:101D500018E3C1E4D0E0CE0176D2F80181938F017F
:101D60002196CB35D105B9F7789480914D38809381
:101D7000473880914E388093143880914F38809343
:101D800011388091503880930E388091513880936B
:101D9000153880915238809312388091533880934F
:101DA0000F3880915438809316388091553880933D
:101DB000133880915638809310388091573880932B
:101DC0001A388091583880934838809159388093D8
:101DD000463880915A388093193880915B388093C7
:101DE0004A3880915C388093493880915D3880937F
:101DF0000B3880915E388093093880915F388093EA
:101E00000A388091603880930838809161388093D7
:101E10000C388091623880931C38809163388093AD
:101E200085388091643880931D388091653880931F
:101E30000D38809166388093403880914A388111FE
:101E400080931B3861E070E08EE496E00E948D057F
:101E5000442443945524539447E0242ECC24C39423
:101E6000D12C65E0362E7CEF672E73E0772EE8EEFE
:101E70008E2EE3E09E2EFEE4AF2EF6E0BF2E0E94F3
:101E80001E018091703890917138009751F06091E7
:101E90006E3870916F380E94A505109270381092BC
:101EA000713880916A38882309F45EC080E00E940E
:101EB000B60140925201809151018111FCCFF9E5A8
:101EC000F0935001809100068E7F809300060E945F
:101ED00081018111FCCF0E9459018091120481601F
:101EE000809312041092943810926D3810926C38CE
:101EF00080916A38882331F180915000897F846015
:101F000080935000809150008160809350008895AC
:101F1000809150008E7F8093500080916C388111A9
:101F200010926A3880919438882331F050921E388C
:101F3000509289380E945F0380916D388823C1F2E6
:101F4000E1DAD6CF22E020931E3880911204887FF8
:101F500080931204BCDA40925201809151018111A8
:101F6000FCCF31E43093500167DB10924C38809104
:101F7000833890918438E2E0853B9E0779F4CCE782
:101F8000D0E0FE018491805394DB8CE291E05DDB34
:101F90002196F0E0C838DF07A1F7C6C02BE08D3AE4
:101FA000920779F03DE08533930709F0B2C0809144
:101FB0003F38813009F0F4C080913E38882309F41D
:101FC000EFC0C0910B38C23011F120F0C43009F4D9
:101FD00083C055CFEC2FF0E0E75FF74CD08186E966
:101FE0000E94B601C11109C0DA3220F4C301019781
:101FF000F1F707C081E090E003C08D2F869590E057
:1020000024DB80E00E94B6018D2F90E0C7C00E94C3
:102010008A018F73E82EF12C0E948A01622DD1D0A3
:10202000E60102C0CC0FDD1F9A95E2F70E948A01FB
:10203000632DC7D0F60102C0EE0FFF1F9A95E2F79D
:10204000CE0FDF1F0E948A0190E0BE01DAD0C80FD8
:10205000D91FC739D10514F0C6E9D0E08C2F0E94F2
:10206000B601C701F2DA8E0133E0159507953A956E
:10207000E1F7011101C001E010E0C701E6DAC01B81
:10208000D10BD7FF02C0C0E0D0E08C2F0E94B60178
:102090000E948A01837039F4C701D7DACE01959581
:1020A00087950E94B601C230D1053CF70E948A0193
:1020B0006DE087D0E60102C0CC0FDD1F9A95E2F7F4
:1020C0000E948A0190E0BE0188D0C80FD91F80E02D
:1020D0000E94B601CE0162C0C0910838CC0FC7394A
:1020E00008F0C6E9D4E08C2F0E94B60185E090E0AC
:1020F000ACDA809108380E94B60181E490E0A5DA5C
:10210000D15089F780ED92E0A0DA80E00E94B6011C
:10211000B6CEF6E084319F0781F480918838ECDAFE
:1021200080911A38882381F0A0927038B09271386B
:1021300010926E3810926F38A2CE26E08433920748
:1021400031F480918638D8DA88EE93E027C035E004
:102150008B3E9307C1F480916B38811190CE8091B2
:102160001B380E94B60184E690E06FDA80E00E949E
:10217000B60120910C38289DC001299D900D112495
:10218000845691090BC0835B954051F480E0CADA14
:1021900081E0C8DA80E0C6DA80ED97E056DA6FCEEB
:1021A00080915000897F8093500080915000816021
:1021B000809350008895809150008E7F80935000CE
:1021C0005ECE991B79E004C0991F961708F0961B04
:1021D000881F7A95C9F780950895AA1BBB1B51E10A
:1021E00007C0AA1FBB1FA617B70710F0A61BB70B87
:1021F000881F991F5A95A9F780959095BC01CD012C
:10220000089597FB072E16F4009406D077FD08D0AA
:10221000E4DF07FC05D03EF4909581959F4F08952B
:10222000709561957F4F0895A29FB001B39FC00143
:10223000A39F700D811D1124911DB29F700D811DF2
:102240001124911D089503D0808199270895FC01E0
:10225000E050FC4E0895262FFADF0080021611F0A0
:1022600004D0019701970895262FAF93BF93E0E024
:10227000F0E1328131FDFDCFDC01A050BC4E2C934A
:102280002DE924BF23E020830196BF91AF910895EB
:04229000F894FFCFF0
:10229400143811380E38000102010000000000005B
:0622A40001000000000033
:1022AA00060B18010101000441294303020D01072D
:1022BA0005787896010A0A78010101412D07020082
:00000001FF
